:020000040000FA
:100000006400EF20850142282034203420344F340E
:100010007634653472342034523461346E3467344B
:100020006534203420342034003420346E34463497
:100030000034203470344634003420346D34483475
:1000400000342034753448340034203443342034B0
:100050003D342034003420344C3420343D342034BA
:100060000034203420342034433461346C34693417
:10007000623472346134743469346E3467342034D9
:100080002034003485148601D120E520061B552834
:10009000F8200B1D4E2804307F20452890012808A9
:1000A0008F0029088E001121452831307F20F8204B
:1000B0009120F8202808A4002908A5008510912087
:1000C000F8202808A6002908A70085149120E5201B
:1000D000F820280803196E280B1D712804307F2092
:1000E0006728CF21CD21861F7A2825307F20B8218F
:1000F0001A2167282B307F20BC214D216728B000B2
:1001000030088820FF3903198A289D20B00A8028EA
:10011000820000000800FD30A1006630A200962891
:10012000922092207E30A1002030A200A20F9628BB
:10013000A10F962800340F39303EAE03031DA428CA
:10014000AF00061EEC202F088515A300230EA92062
:1001500023080F3986000515000005114230A10063
:10016000A10BB028003418309F00AA01AB01AC01EC
:10017000AD012A3084000430A0003330800780199C
:10018000F039801B0F398002840AA00BBD288E0D28
:100190008F0D900DAD0DAC0DAB0DAA0D9F0BB928B9
:1001A00008009220851105110330A9209220033008
:1001B000A9200330A9200230A9200C30ED202830DE
:1001C000ED200630ED200130E8280930AE00023085
:1001D000EA208B288511A528C030EA20AE28831696
:1001E0003730810010308500F0308600831208001F
:1001F0000B1181010514A801A90183161130850096
:1002000092201030850083120108A8008316011681
:10021000000001128312A903010828060319062908
:100220000800B3207C217E21802182218421862127
:1002300088218A292A080F39031924299B20802123
:1002400082217A21842137292B0E0F3903192E2977
:100250009B2082217A218421862137292B080F397E
:10026000031939299B207A21842186218821153080
:100270007F282C0E0F39031D462920309D202C0885
:100280000F39031D472920309D20482984218621CC
:1002900088217A218A2119307F282A080F390319E9
:1002A00057299B2080217A218221842160292B0ECD
:1002B0000F39031962299B207A218221842186210A
:1002C0001D307F282B080F3903196C299B208421AE
:1002D00086217A21882178292C0E0F39031D732954
:1002E00020309D207429842186217A2188218A2129
:1002F00021307F282E309D282A0E9B282A089B28F3
:100300002B0E9B282B089B282C0E9B282C089B2807
:100310002D0E9B282D089B287F23912907239129A7
:10032000B7221C0895001D0896001E0897000800BB
:1003300015089C0016089D0017089E000F089500E0
:10034000100896001108970008000F08B000150863
:100350008F00300895001008B00016089000300893
:1003600096001108B00017089100300897000800A7
:100370008E21DE219021C4299021D7219021EC21CA
:1003800098219021A5218E21901FC8292D30C9299F
:1003900020309D2090135B22B328F021D029EE213C
:1003A000EC218E2198219021E621A5218C299821EC
:1003B000AB309100383090004D30E42998218C30DA
:1003C00091001C30900040308F000800982191016E
:1003D00090018F010130F9292430F1292630F129CB
:1003E0002830840098219101900100088F00840A30
:1003F00000088E001A2A9B011008031D052A0F0809
:1004000090000319152A8F019B151B089102031DEB
:10041000031C732B0310901B122A8F0D900D910B50
:100420000B2A732B921F9013003490018F018E01C1
:1004300091010034963091009201901F282A8E0974
:100440008F0990098E0A03198F0A0319900A9217CF
:100450009B011008031D3D2A0F0890000E088F0015
:100460008E019B151008031D3D2A0F0890008F0177
:100470009B111B1610080319152A1B089102031D56
:10048000031C732B0310901B4B2A8E0D8F0D900DA8
:10049000910B432A732B131B0F1C122A8E1F122A37
:1004A0008F0A0319900A031D122A900C8F0C910ACF
:1004B0000319FD2A122A8E011108031900341008AD
:1004C0009200901796309102911FAB2A9109910AE0
:1004D00008301102031C872A91008E0D0F088E0030
:1004E00010088F00900108301102031C872A910028
:1004F0008E0D0F088E008F0108301102031C872A11
:1005000091008E0D8E011108031D0310902A110811
:100510000319902A0310900C8F0C8E0C910B8A2AD1
:10052000131B0E1C9C2A031C9C2A8E0A03198F0A7B
:100530000319900A901BAB2A921F003490098F096F
:100540008E098E0A03198F0A0319900A003490014C
:100550008F018E0100341314931FFF349001921FFA
:10056000FF3090008F008E00920D900CFF34110828
:10057000031D17080319152A1008160692001708FC
:1005800091077E30031CC82A91020318FD2ACB2A4A
:100590009102031C732B10088E000F088D008E171C
:1005A0009617031090018F0110309B000D1CDE2A5E
:1005B00015088F0716080318160F9007900C8F0C5C
:1005C0008E0C8D0C03109B0BD62A901BEB2A8E0DE4
:1005D0008F0D900D9103131B0F1CFA2A8E1FFA2A00
:1005E0008F0A0319900A031DFA2A900C8F0C910AA6
:1005F0000319FD2A921F901300349314931FFF34A4
:10060000FF30910090008F00920D900CFF3417087E
:1006100003197D2B11080319152A100816069200DC
:10062000901796179B0110088E000F088D00150873
:100630008D021608031C160F8E028E018D01031CFD
:10064000272B0310900C8F0C8E0C01309B00170889
:100650009102031C312B7E301B0791070318FD2AE2
:10066000362B7E301B079107031C732B10309A002A
:100670008D0D8E0D8F0D900D9B0D15088F02160898
:10068000031C160F9002160D9B041B1C492B0D1406
:10069000502B15088F0716080318160A90070D101F
:1006A0009A0B382B131B0D1C6C2B03108F0D900D08
:1006B0009B0D15088F021608031C160F9002160DCD
:1006C0001B0401398D0703188E0A031D6C2B8E0C39
:1006D0008D0C910A0319FD2A921F8E130E089000AB
:1006E0000D088F0000341315931FFF340130910063
:1006F00090018F01920D900CFF349315FF348030E0
:100700009606100816069B008E0194011108170228
:10071000031C9C2B17088C00110897000C089100F3
:1007200016088C00100896000C08900015088C0024
:100730000F0895000C088F001708031900341008E3
:100740009200901796171708110297000319C22BF1
:1007500008301702031CB92B9700150894001608DF
:100760009500960108301702031CB92B120890005F
:10077000003417080319C22B0310960C950C940C27
:10078000970BBC2B9B1FCC2B940995099609940AB7
:100790000319950A0319960A14088E0715080318F9
:1007A000150F8F0716080318160F90079B1BE02BD9
:1007B000031C4B2A900C8F0C8E0C910F4B2AFD2A98
:1007C0000318282A8E098F0990098E0A03198F0AA7
:0A07D0000319900A80309206FB29FD
:02400E00F23F7F
:00000001FF
